:020000040000FA
:10000000000000000000052809005C21851424215F
:10001000A40057200628A201A3000310230D820785
:100020001A20142838201428FF39031908005621F3
:10003000A20A0D2822088207433420343D3420349C
:1000400043346134733473346534743474346534D4
:10005000203474346F342034503443342C342034FE
:10006000423461347534643420343D3420340034F7
:1000700022088207503420343D3420345034433435
:10008000203474346F342034433461347334733423
:10009000653474347434653473342C34203442340D
:1000A00061347534643420343D3420340034240801
:1000B000433A031964202408503A03196F20240896
:1000C000473A03197A2008002408B1004E21003075
:1000D0000B2006212808303E56214E210800240816
:1000E000B1004E2101300B2006212808303E562158
:1000F0004E2108003108433A0319BD203108503A17
:1001000003196E2108006030A200FF30A300013007
:100110008E20A30B8728A20B85280800A100AC30F5
:10012000A00000009328A00B9128A10B8F2801307C
:1001300085060800B000B5200830B500B00C031CDF
:10014000A328AC20A428B520B50B9E28AC200630EF
:100150005621AC20242108002808A90001308E2057
:1001600001308E20A90BAE2808002808A900A9009C
:1001700002308E20A90BB82808008510DA2030083C
:10018000533A0319CB283008393A0319CF283210D3
:1001900030085621BD28321430085621BD283218A7
:1001A000D528321030085621BD2830085621FF309E
:1001B000562108002808A900F2200318DC28A90B02
:1001C000DC287F30B0002808A900F220A90BE52820
:1001D000B00C0318E3282808A900F220A90BED2889
:1001E00030080800810106080B100B1CF5280608D2
:1001F0000B1001088101603C031C08000B1CFE2849
:1002000006080B1001088101603C08002421A800A9
:10021000383A031D0E290830A80008002808343A8F
:10022000031D15290430A80008002808323A031DD0
:100230001C290230A80008002808313A031D232990
:100240000130A800080006298C1E24291A088C12E7
:100250000800831203138316871707130A309900C7
:10026000243098008312903098000800A5004121A6
:10027000A600250E4121A700270856212608562151
:1002800008000F39A000A1000A30A102A11F4B29CC
:100290002008303E08002008373E08000D30562167
:1002A0000A3056210800FF30562108008316981C9A
:1002B0005729831299000800831203138B132921F5
:1002C000831603308100FF30860006309F00003027
:1002D0008500831200309F0085140800851083205C
:1002E00006305621AC202421B0009A20B000B01F67
:0802F000752983208514080024
:02400E00723D01
:00000001FF
